:101A400023475F485F3330232020202020202020A0
:101A500023424C48454C492445464D3842323123B7
:101A0000100521FFFFFFFFFFFF09FF01FF55AA019E
:101A1000FFFFFFFFFF03FFFFFF25D0285004FF0259
:0A1A2000FF7AFF0701FFFF0000FF3F
:101A60002020202020202020202020202020202076
:030000000219FDE5
:030003000202EC0A
:03000B0002008D63
:030013000204FFE5
:03001B0002009050
:03002B000202B618
:03005B0002050E8D
:030073000202D9AD
:100080000406080C10182030406080A0C0054032E3
:10009000C2AFC2A853E6EFC28E85698BC0D0D2D35F
:1000A000C0E0C0F0C2CAA8CCA9CDD2CAD2AF758A6E
:1000B00000C3E8956AF8E9956BF9C3E913F9E81309
:1000C000F8E5646007C3E913F9E813F8E97025E877
:1000D000956C4020956C501CE582B410177C007B19
:1000E000007A007908900000A868E5647004C3E80D
:1000F00013F801FD900000D2A8D2AA61B7E0FDC3B9
:100100009CC39840EF98EB33FB0582E0FCC39DC392
:100110009840E198EB33FB0582E0FDC39CC3984017
:10012000D398EB33FB0582E0FCC39DC39840C59890
:10013000EB33FB0582E0FDC39CC39840B798EB33DB
:10014000FB0582E0FCC39DC39840A998EB33FB05F7
:0D01500082E0FDC39CC398409B98EB33FBFD
:10015D000582E0FCC39DC398408D98EB33FB05826F
:10016D002178900000D2A8D2AA61B7E0FDC39CC34C
:10017D009840EF98EA33FA0582E0FCC39DC398409E
:10018D00E198EA33FA0582E0FDC39CC39840D39809
:10019D00EA33FA0582E0FCC39DC39840C598EA3363
:1001AD00FA0582E0FDC39CC39840B798EA33FA057F
:1001BD0082E0FCC39DC39840A998EA33FA0582E01A
:1001CD00FDC39CC398409B98EA33FA0582E0FCC3BB
:1001DD009DC398408D98EA33FA0582EBC46B6A543F
:1001ED00F0F9EAC454F0C3996009900000D2A8D286
:1001FD00AA61B7EBF4C454F0F9EAF4C4540E49FA09
:0B020D00EBF4C4540FFBC3EA9460FA4A
:10021800EB9400FB50067B007A007900303A27C344
:10022800EA94D0F8EB9407F9400BE8FAE9FB20359B
:1002380009D2354142303502C235203902B235C3C0
:10024800EA33FAEB33FBEB2B3B3BF9C3EB13FBEA4B
:1002580013FAEA29FAEB3400FB30E3047AFF7BFF58
:10026800E5255403601B202A18E55B33F9EB70077A
:10027800C3E99A4002E9FAE53CC4332AFAEB3400B0
:10028800FBC3EA33C4540FF8EB33C454F048F87096
:1002980005EA60027801900000D2A8D2AAE522609F
:1002A80002152281A4900000D2A8D2AA61B7C0D0BA
:1002B800C0E0C2CF0541E5646009E5636005756388
:1002C8000041D4756301E52360021523D0E0D0D046
:1002D80032C2AF53E67F7592FA7593FFC2205391ED
:1002E8007FD2AF32C0E0E58A30340885698BF0A34D
:1002F800D0E032D0E0C2AF53E6EFC0D0C0E0C0F0EB
:0D030800D2D3D2AF5388EFA88AA98CAA40A7
:10031500308D010A758A00758C0075400043881080
:10032500E564700AC3E833F8E933F9EA33FA3033A0
:100335001FE8C4540FFAE9C454F04AFAC3132AFA61
:10034500C3E833F8E933F9E82AFAE93406FB61A88A
:1003550030320FC3E833E933FAE82AFAE93400FB0F
:1003650061A8303115E875F056A4AAF0E975F05684
:10037500A42AFAC5F03400FB61A8C3EA13FAE9130D
:10038500F9E813F8E875F056A4AAF0E975F056A453
:100395002AFAC5F03400C313FBEA13FAC3EB13FBC7
:1003A500EA13FAC3EB94125009C3EA9434EB9407A9
:1003B50050160522E52270021522C3E5229432501B
:1003C5000281F275520081F5E52260021522303670
:1003D500067C007D0861E7AC31AD32303A04AC33C0
:0D03E500AD34C3EA9CFAEB9DFB9208AE5EBE
:1003F200AF5F303A425007203509D235810530359A
:1004020002C235303504AE60AF61203902B235C365
:10041200EA33FAEB33FBA208500AEAF42401FAEBBE
:10042200F43400FBC3EA9450FAEB9400FB501478C6
:10043200007A007B008145A208500878007A007B90
:100442000081A4E5255403601B202A18E55B33F9DB
:10045200EB7007C3E99A4002E9FAE53CC4332AFA91
:10046200EB3400FBEA8EF0A4F9AAF0EB8EF0A42A9A
:10047200FAC5F03400FBC3EB13FDEA13F8C3ED1326
:10048200FDE813F80FEF146004C3E833F8C3E9334F
:10049200EA33FAEB33FBDFEDEB30E30678FF7AFF6A
:1004A2007B078852D230C3E559FC955A4002AC5AB8
:1004B200C3EC95525008EC75F008A4FAABF0EAF4DC
:0C04C200F8EBF45407F9C3E8943CFAE9A5
:1004CE009400FB50047A007B00885489558A568B21
:1004DE005775230AD0F0D0E0D0D053F7DF43F74062
:1004EE0043E6103275230AD0F0D0E0D0D043E610A8
:1004FE0032C2AAD28EC2CA85CC6A85CD6BD2CA321E
:10050E00C2AFC0D0C0E0D2D3A8F9E55830E20AE5B8
:10051E00FA20E24C20E149A12FE5FA30E24220E137
:10052E003FC3E55513F8E55413F5FB88FCC3E557B7
:10053E0013F8E55613F5E988EA85555853F7BFD2F7
:10054E00A8303402D2AA53E6EFC3E5529401400517
:10055E00755300A16EE5532401F55350037553FFF7
:10056E0053F7DFD0E0D0D0D2AF32790180147903C7
:10057E008010790A800C791E80087964800479C80D
:10058E0080007817E4D5E0FDD8FAD9F6227A147BEC
:10059E007880127A107B8C800C7A0D7BB480067A70
:1005AE000B7BC88000E562D5E001227902E4C2939C
:1005BE00D5E0FDD292D5E0FDC292D5E0FDD293D525
:1005CE00E0FDE920E002D29030E002D294E562D55F
:1005DE00E0FDE920E002C29030E002C2947496D5AC
:1005EE00E0FDD9C9EAF8D5E0FDD8FBDBB8C293220D
:0705FE0078FF20282879A1F5
:10060500E76023E548601F74FF8548F084853FF067
:1006150030290375F005A4F8C5F0600278FFC3E83A
:10062500955B5002A85B885A22C3E54794A0E5482C
:100635009400E55A500314C13F046002F55A22752F
:10064500E89022055CC3E55C9408405330EDF4A8BE
:10065500BDA9BE755C00E9FA79A0E76041EA7006BC
:10066500E55D6018800CC3E8955D600EE55D50059D
:10067500600A1480070460FA8002E55DF55DC395A4
:1006850067401B7559C0C394044013755980C394C2
:1006950004400B755940C39404400375590022E585
:1006A500592410500274FFF55922743279A687F047
:1006B500A4C5F0A2F733F8C3E895594002A85988B4
:1006C5005B227547007548F022C2AFC2CAA8CCA903
:1006D500CDAA4130CF010AD2CAD2AFC3EA13FAE993
:1006E50013F9E813F8AB42AC4388428943C3E89B4E
:1006F500F8E99C20280A547FF9302C02E1ECE14509
:06070500AD448A44F9EA4C
:10070B009D547FFA600678FF79FFE12AAE45AF462C
:10071B008B458C46A842A943C3E89EF8E99FF9C3D1
:10072B00E54813FBE54713FAE82AF547E93BF5489B
:10073B0050067547FF7548FFE192AA47AB48AC4797
:10074B00AD487E047F02C3EB9404400D1E1FC3EB28
:10075B00940840052029021E1FC3ED13FDEC13FC6A
:10076B00DEF7C3EA9CFAEB9DFBEF6009C3E913F9D3
:10077B00E813F8DFF7EA28FAEB39FB8A478B485086
:10078B00067BFF8B478B48C3EB94025002D22C3075
:10079B0028047F03E1BD7892E6FFC3E53D948240D8
:1007AB00110FC3E53D94A040010FC3EF9406400227
:1007BB007F057E02E548C4540FF9E548C454F0F8B0
:1007CB00E547C4540F28F8C3E89EFAE99400FB40B0
:0E07DB0009C3EA9401EB940050047A01E4FB98
:1007E900020838AA47AB48EBC4FEEAC4540F4EFCD2
:1007F900C3EA9CFAEB9400FBC3E813C313F8EA2895
:10080900FAEB3400FB8A478B48C3EB94024002C2DF
:100819002C7802EBC4FE7B00EAC4540F4EFAC3EAFB
:1008290098FA4005C3940150027A017892E6FF30A4
:1008390020020138854E92854F93D22043E680C32A
:10084900E49AF8E49BF9C3E833F8E933F9302C0367
:100859000208CDE8FAE9FBD3E913FDE813FC884E59
:10086900894FC3EF94036038EF20E00CE82CF8E9D6
:100879003DF9ECFAEDFB8013E828F8E939F9C3E80A
:100889002401F8E93400F97AFF7BFFC3EF940340B0
:100899000F8A508B51884A894B8C4C8D4D02090225
:1008A900885089518A4A8B4B8C4C8D4D3028127552
:1008B90050F07551FF754CF0754DFF754EF0754F41
:0108C900FF2F
:1008CA00020902E8FAD3E813FC884EC3EF940360E6
:1008DA0021EF20E007E82CF8ECFA01EDE8282401E2
:1008EA00F87AFFC3EF940340098A50884A8C4C0275
:1008FA00090288508A4A8C4C3020022102753A0239
:10090A00D22043E680E5255403602DA847A948C3B1
:10091A00E913F9E813F8302804E92440F9C2AF537F
:10092A00E67F759100C3E498F594E499F59575917D
:10093A0004D22043E680D2AF22D221754900752025
:10094A0000302B037520402161D2217549007520A2
:10095A0040302B0375200078017901202C20E525F1
:10096A0054036002C2217914E548C313700104F8E4
:10097A00C3941440027814302804781B791BC3E806
:10098A0033F8C3E933F9202010E549600C30280315
:10099A00D53A04D2234114310A0549E59B5440B59E
:1009AA00200221FE30280908C3E899400118219045
:1009BA0020210A08C3E899400221612190C22153EB
:1009CA00E67F759100302C117594007595F075913C
:0609DA0004D22043E68078
:1009E000020961E5487EFFC3334009C3334005C3B4
:1009F000334001FEC3E49E759400F59521D8C3E50C
:100A0000399401500221613021022161D802411242
:100A10002190C223C2AF53E67F7591008550948523
:100A20005195759104854A92854B93D22043E68077
:100A3000D2AFE52554036007202902053980103024
:100A4000230D202B0A202107158115810211F42284
:100A500078003021027801E53D75F007A4F9E5F052
:100A600028F5F0E9A2F013A2F113A2F213F53DC3A9
:100A700094785003753D78C3E53D953E400BD222F6
:100A8000C290C292C29475D53F3020024189854CF4
:100A900092854D93D22043E68022203810C2AFC207
:100AA00093D29175D52FD2AF759F03616AC2AFC241
:100AB00093D29575D53ED2AF759F03616A203810E9
:100AC000C2AFC29475D53BD291D2AF759F13616A04
:100AD000C2AFC29075D53BD295D2AF759F23616AE4
:100AE000203810C2AFC291D29575D53BD2AF759F59
:100AF000238077C2AFC295D29175D53BD2AF759F97
:100B0000138067203810C2AFC29275D53ED295D2FD
:100B1000AF759F038054C2AFC29275D52FD291D2C8
:010B2000AF25
:100B2100759F038044203810C2AFC295D29375D50A
:100B31003ED2AF759F138031C2AFC291D29375D5AA
:100B41002FD2AF759F238021203810C2AFC290757C
:100B5100D52FD293D2AF759F23800EC2AFC29475A9
:100B6100D53ED293D2AF759F13C22222C290C292B8
:100B7100C294C291C293C29575D53F22788076FF07
:100B81000876FF0876FF0876FF0876FF0876FF08EB
:100B910076090876FF087601788C76010876FF08D9
:100BA10076FF0876FF0876FF0876FF087603087659
:100BB100FF0876FF0876FF0876250876D0087628A4
:100BC1000876500876040876FF0876020876FF0852
:100BD100767A0876FF0876070876010876FF0876A8
:100BE100FF08760008760022FA75F00CA4ABF0EA53
:100BF100C333F8740133F9E8C333F8E933F9E8C3CF
:100C01002BF8E93400F9E8C333F8E933F92278889D
:060C1100E6C39403D23A91
:100C17005002C23AC238E630E102D238A2389239DD
:100C27007886E6149000809378A6F67886E6F53FF6
:100C3700C394025003753F02789CE6753EFFB402E9
:100C470003753EA0B40303753E8278A0E6F86006FC
:100C570074282409D8FCF5677896E671E988318904
:100C670032789EE671E9883389347897E671E988A6
:100C7700358936716D223036117A007B007CFF7D15
:100C8700007E0091E38B5F8A5E22303A227896E6F7
:100C9700FA7B00789EE6FC7D00C3EA33FAEB33FB70
:100CA700C3EC33FCED33FD7E0A91E38B618A6078F8
:100CB70096303A02789EE6FA7B007897E6FC7D004C
:100CC7007E00303A10C3EA33FAEB33FBC3EC33FC54
:100CD700ED33FD7E0A91E38B5F8A5E22C3EC9EFCB7
:100CE700ED9400FDC3EC9AFCED9BFDC3EC9423ED62
:100CF700940050047C237D00C3EC94FFED940140E5
:010D070004E7
:100D08007CFF7D017BFF0B7A000AEA7009C3EC3394
:100D1800FCED33FDA10EEC8AF0A4AEF0ED8AF0A450
:100D28002E947C40E4EAF460DD22D236917D1205EF
:100D3800841205847A007B007C1012057CE5522A17
:100D4800FA74003BFBDCF37C04C3EB13FBEA13FAF5
:100D5800DCF7FFEB60027FFFC236917D2278A5E6C3
:100D6800F954037000E9540C7000E954307000E93C
:100D780054C07000227565007566007597DE75971A
:100D8800AD7581C043FF8075EF0675A900716D755B
:100D980080FF75F1F075A4007580FF75D4FF75901C
:100DA8000075F23F75A53F75900075D53F75A60192
:100DB80075E34075E202716DE4F8F6D8FD717D12B5
:100DC800123878988662753001C2AF12058C120508
:100DD8009B1205841205A11205841205A712058429
:100DE800B165C2AF75650075660078FA79FA308525
:100DF80007D9FBD8F7021C00910F917D789886627D
:100E0800716D75A91375A71075C10075A700756474
:100E18000075E405758811758E0475890975C8040F
:100E280075910475D84075D90875F782759E037554
:0B0E3800960275DA4275DB0075A823F6
:100E430075E69075B801759B80759D0075D10C751D
:100E5300BCB975BB1075E88075B201120578D2AFC5
:100E6300753C00C23012058CC231C232C233C23467
:100E7300752200120588C3E522940A5002E138D294
:100E830031752200120588C3E522940A5002E13825
:100E9300C231D232752200120588C3E522940A506A
:100EA30002E13875E4D5758851758E017589AA7587
:100EB3008C00758D00C2A9D2ABD2AA756980756802
:100EC30014756C50C232D2347522001205887568CD
:100ED30010C3E522940A405D758E0C756900756830
:100EE30028756C28752200120588756820C3E522D1
:100EF300940A4041758E0C756980756814756C147D
:100F0300752200120588756810C3E522940A4025EE
:100F130075E405758811758E04758909D2A9C2AB6C
:100F2300C2AAC234D233752200120588C3E52294C3
:100F33000A4002A1EA12057C203003020DEAC2AF87
:100F430012059B12059B12059BD2AF12058C203410
:100F530003303A03020FFC12057C788CE6C394013C
:100F63005002E1FCE530C394015002E1FC7565A534
:100F73007566F17F02D236917D120588C2AFC23603
:100F8300917DC3E552947FD2AF406E120578C2AF14
:100F93001205ADD2AFDFDEB132C3EF7897F612059B
:010FA3008CC1
:100FA4001213267F0AD236917D120588C2AFC2364B
:100FB400917DC3E552947FD2AF50E8120578C2AF59
:100FC40012059B12058012059BD2AFDFD8B132EF18
:100FD40024037896F6F87997E7C39423400398504E
:100FE40006E824237897F612058C12127F12135503
:100FF400120588917D020DEA75650075660012057B
:1010040088C3E55294014003020F51C2AF1205ADEB
:101014001205AD1205ADD2AF12058C753000E4F5A2
:1010240037F5380537E537F4703F0538789AE678B0
:1010340019146012783214600D787D14600878FAFF
:10104400146003753800C3E53898401D120B6D1207
:101054000578153875370078998662C2AF1205ADE8
:10106400D2AF78988662120588120580E523700352
:10107400020DEAC3E552940140A9120588E52370E4
:1010840003020DEAC2AF120B6DE4D2AFE4F55CF5D6
:1010940024F525F53D755C0812057812064430EDFB
:1010A400FDA8BDA9BEE97001F8885D120648755C0B
:1010B40008C2AF7559FF1206AF855B59855B5AD2DA
:1010C400AF75A71075C13075A70075A903756401C4
:1010D400303A07C238303502D238D2287539001276
:0810E4000B26120B491206C78E
:1010EC001206CE1206C71206CE1206C712095312EA
:1010FC000A50120A9A1206CE120943202C0312052A
:10110C00FE302C0312062E120A50120ABD1206CE05
:10111C00120953120A50120AE01206CE1209431297
:10112C000A50120B031206CE120953120A50120B5C
:10113C00261206CE120644120943120A50120B490B
:10114C001206481206CE302827855B5979187A0C7E
:10115C00C3E53999400EC228D2298A3B855B598553
:10116C005B5A800CC3E552940140030210F821FC39
:10117C0030291C202B19E53B147006C229D22A01F8
:10118C00F8F53BC3E552940140030210F8806175F9
:10119C003C0078FA79A4E760027803C3E5539850D1
:1011AC004FE523604B303A17203805203507800F68
:1011BC00303502800A202B07D22B855B59212878E9
:1011CC00F0302B05855B597820C3E5489850030215
:1011DC0010F8302B1BC22BC238303502D238D22932
:1011EC00753B12855B5901F8053CE552600221FF05
:1011FC00753C00C2AF120B6D75240075250075A9E6
:10120C001375A71075C10075A700756400D2AF12D5
:10121C000588120B6D78A4E66006D291D293D29514
:10122C00C3E53C94044003020DEA0122901A0D78A8
:10123C002051B9E520B4550AA351B9E520B4AA024E
:10124C0080137565A57566F1120B7D517F75650070
:10125C00756600801D901A0378807B0A51B9A3082B
:10126C00DBFA901A0F788C7B1A51B9A308DBFA9031
:10127C001A2922C2AF1212FC51D9901A00741051C3
:10128C00BEA3740551BEA3742151BE901A0378807D
:10129C007B0A51BDA308DBFA901A0F788C7B1A518C
:1012AC00BDA308DBFA710F51ED901A2922E493F6D5
:1012BC0022E6438F01538FFDFFC3E583941C40014D
:1012CC0022EF8565B78566B7F0538FFE22438F02F8
:1012DC00438F018565B78566B7901A0DF0538FFC67
:1012EC0022901A0D745551BE901A0E74AA51BE223A
:1012FC007A3079D07820901A4051B9E520F709A3BB
:10130C00DAF7227A3079D0901A40E751BE09A3DA85
:10131C00F9227C0512058CDCFB22C2AF12059B1254
:10132C0005A11205A71205AD12058012059B120529
:10133C00A11205A71205AD12058012059B1205A17D
:10134C001205A71205ADD2AF22C2AF1205AD120520
:10135C00A71205A112059B1205801205AD1205A757
:10136C001205A112059B1205801205AD1205A712DC
:08137C0005A112059BD2AF226E
:101C0000C2AFC2D37597DE7597AD7581C075A90057
:101C100043FF80752438752503B1DB7529A5752A26
:101C2000F143F12053A4DFD28575D4FF75E3407DE5
:101C3000FA780379E67C10752200752300901DE880
:101C40007B0675249875250130850281482085081A
:101C5000D8FBD9F9DCF781BA308508D8FBD9F9DC93
:101C6000F781BAB19BE493A3C39A6004DDC381BA40
:101C7000DBDBB18D600281317B08E493FAA3B16EA6
:101C8000DBF87A30B16E752200752300B18DEAFC65
:101C9000EBFDC3ED94FE400EB18D8A278B28ED300D
:101CA000E0048A828B83B18D7AC270D8C3ED94FE32
:101CB000601950CEBD0029EC600F7520007521FF22
:101CC000752900752A000200008100A827A92808AC
:101CD00009D804D90281DDB191EAF281D10D81A642
:101CE000C3ED94035051EDA2E092007AC5C3E582A2
:101CF0009400E583941C508C200010438F02438F86
:101D0000018529B7852AB7F0300027A827A9280818
:101D100009438F01538FFDD804D902A132C3E58353
:101D2000941C4003A3A117E28529B7852AB7F0A325
:101D3000A117538FFC81827AC1BD030CE493A3FAEF
:101D4000B152DCF8B14A81828184AA22AB23B16E00
:101D5000EBFAEA6222752608C3E52313F523E52290
:101D600013F52250066323A0632201D526EAB1DBD6
:101D7000B1DB75260AEAF4200102D285300102C2E5
:101D800085B1DBC3134002C201D526EB22B191EA33
:101D9000FB208502A191308502A196752608AE240C
:101DA000AF25C3EF13FFEE13FEB1DFB1DBC3EA13C0
:101DB0003085024480FA30E703632201C3E5231330
:101DC000F523E52213F52250066323A0632201D5F3
:101DD00026D9E52265236523F52222AE24AF250E00
:101DE0000FDEFEDFFCD20122424C48656C693437BD
:061DF0003164E8B20601B7
:0319FD00020D7D5B
:00000001FF
